S02B0000433A2F576F726B2F736F6674776172652F4F70656E424C542F5461726765742F44656D6F2F41524DEF
S31508000000E011002051010008F50E0008F50E000861
S31508000010F50E0008F50E0008F50E0008F50E0008A6
S31508000020F50E0008F50E0008F50E0008F50E000896
S31508000030F50E0008F50E0008F50E0008F50E000886
S31508000040F50E0008F50E0008F50E0008F50E000876
S31508000050F50E0008F50E0008F50E0008F50E000866
S31508000060F50E0008F50E0008F50E0008F50E000856
S31508000070F50E0008F50E0008F50E0008F50E000846
S31508000080F50E0008F50E0008F50E0008F50E000836
S31508000090F50E0008F50E0008F50E0008F50E000826
S315080000A0F50E0008F50E0008F50E0008F50E000816
S315080000B0F50E0008F50E0008F50E0008F50E000806
S315080000C0F50E0008F50E0008F50E0008F50E0008F6
S315080000D0F50E0008F50E0008F50E0008F50E0008E6
S315080000E0F50E0008F50E0008F50E0008F50E0008D6
S315080000F0F50E0008F50E0008F50E0008F50E0008C6
S31508000100F50E0008F50E0008F50E0008F50E0008B5
S31508000110F50E0008F50E0008F50E0008F50E0008A5
S31508000120F50E0008F50E0008F50E0008F50E000895
S31508000130F50E0008F50E0008F50E0008F50E000885
S31508000140F50E0008F50E0008F50E0008F50E000875
S315080001502949072291438D4628482949294A00F00A
S3150800016039F8294829492A4A00F034F829482A49F9
S315080001702A4A00F02FF82A482A492B4A00F02AF87A
S315080001802A482B492B4A00F025F82B482B492C4A9C
S3150800019000F020F82B482C49002200F026F82B48BE
S315080001A02B49091A082903DB002202600430016082
S315080001B01C481D49884205D00268043003B490479C
S315080001C003BCF7E700208646EC4600200021214ABA
S315080001D09047FEE7884207D0521A05D003780130C7
S315080001E00B700131013AF9D17047884202D002708A
S315080001F00130FAE770470000E0110020D8510008E6
S3150800020000000020180000205802000858020008C4
S3150800021080450008D8510008000000200000002092
S31508000220804500088045000880450008804500088C
S31508000230804500088045000880450008804500087C
S31508000240D851000818000020600F0020600F002019
S30D08000250E00F00207503000809
S3150800025800B5C7B04FF48C720021684604F05CF903
S315080002686946094803F0A8FF40B9009B43B19DF8C1
S31508000278080080F01000C0F3001002E0002000E03B
S31508000288002047B05DF804FB804500080048704721
S315080002988045000808B50748002380F828320A224E
S315080002A8054903F0F3FB18B90122024B83F8282203
S315080002B808BD00BF18000020A045000870B50E4B01
S315080002C893F82832012B02D10B4803F0ABFE01F054
S315080002D8E5F900F16406094D402403E001F0DEF96A
S315080002E8864205D32146284600F0FAFD0028F5D0AF
S315080002F8034803F087FF70BD18000020004400403B
S315080003088045000808B5044B93F82832012B02D11A
S31508000318014803F087FE08BD1800002070B5064698
S31508000328104B93F82832012B0AD10E4903F0F0FF37
S31508000338002805DA0B48002380F8283203F072FEF5
S31508000348317871B1084C8025204600F0C5FD29464C
S31508000358204600F0C5FD0028F9D016F8011F002927
S31508000368F2D170BD180000200044004000B583B0E3
S3150800037800230093019303F1804303F504331A68B5
S3150800038842F001021A605968554A0A405A601A68C2
S3150800039822F0847222F480321A601A6822F48022C3
S315080003A81A605A6822F4FE025A604FF41F029A60CD
S315080003B81A6842F480321A60194640F2DC520B6811
S315080003C803F400330193009B01330093019B13B98F
S315080003D8009B9342F3D1434B1B6813F4003F03D1A8
S315080003E86E21414801F01EFA404B1A6842F0100285
S315080003F81A601A6822F003021A601A6842F00202A2
S315080004081A60A3F580535A685A605A6842F400522B
S315080004185A605A6842F480625A605A6822F47C1212
S315080004285A605A6842F4E8125A601A6842F08072AA
S315080004381A601A6812F0007FFBD02A4B5A6822F015
S3150800044803025A605A6842F002025A601A4653680A
S3150800045803F00C03082BFAD1224B9A6942F00902D9
S315080004689A61234A516821F00F015160516841F099
S3150800047808015160516821F0F0015160516841F056
S31508000488B0015160A2F54062516821F4C04151603B
S31508000498516841F480415160DA6942F00072DA61C4
S315080004A8DA6942F40032DA619A6942F005029A6119
S315080004B8A3F584331A6822F470621A601A6842F43B
S315080004C830621A601A6822F470421A601A6842F48E
S315080004D880421A6001F0DCF901F0EAF9FCE700BF8E
S315080004E80000FFF800100240B0450008002002404E
S315080004F8000C014038B50146074800F0D3FC064D04
S3150800050801242146284600F0E1FC0028F9D00248D3
S3150800051800F0CAFCC0B238BD0038004070B501F01A
S31508000528BDF800F5FA76FF252846FFF7E3FF0446E7
S31508000538FF2803D001F0B2F88642F5D8FF2C14BF7D
S315080005480020012070BD00BF08B54FF4805103484C
S3150800055800F05AFCFF20FFF7CDFF08BD000C01404C
S3150800056810B54FF48051084800F050FCFF20FFF7FB
S31508000578C1FFFFF7D3FF18B90446FFF7E5FF00E008
S315080005880124204610BD00BF000C014038B50446BA
S315080005980D4610F0800F07D000213720FFF7F6FF29
S315080005A801283AD804F07F04FFF7CEFFFFF7D8FFF3
S315080005B848B344F04000FFF79DFF280EFFF79AFF5F
S315080005C8C5F30740FFF796FFC5F30720FFF792FF25
S315080005D8E8B2FFF78FFFE4B1082C16D00120FFF721
S315080005E889FF0C2C02D1FF20FFF784FF0A24FF2578
S315080005F82846FFF77FFF10F0800F0ED0631E13F012
S31508000608FF04F5D138BDFF2038BD8720FFF772FFF4
S31508000618ECE79520FFF76EFFE8E738BD38B50546DD
S315080006280C46FFF77BFF034618B32046FFF762FF21
S31508000638FD2C1DD0AC1C05F2022514F8020CFFF798
S3150800064859FF14F8010CFFF755FF0234AC42F4D1F0
S31508000658FF20FFF74FFFFF20FFF74CFFFF20FFF7AC
S3150800066849FF00F01F00052814BF0023012300E0F6
S315080006780123184638BD00BFF8B504460D4601F0F3
S315080006880DF800F16407FF263046FFF733FFFF2809
S3150800069805D101F003F88742F6D80020F8BDFE28F0
S315080006A816D10234FF263046FFF724FF04F8020C59
S315080006B83046FFF71FFF04F8010C0234023DF2D159
S315080006C8FF20FFF717FFFF20FFF714FF0120F8BDEB
S315080006D80020F8BD002840F05981B24B1B7813F06A
S315080006E8020F03D0AF4B1878C0B270472DE9F04314
S315080006F889B00121082000F08BFB01214FF48040C6
S3150800070800F094FB4FF48057ADF800704FF01009CD
S315080007188DF8039003268DF80260A34C6946204697
S3150800072800F022FB3946204600F06EFB4FF42043C2
S31508000738ADF800308DF8026018238DF80330694645
S31508000748204600F011FB4FF48043ADF800304823EB
S315080007588DF803306946204600F006FB0025ADF8FB
S3150800076808504FF48273ADF80A30ADF80C50ADF85E
S315080007780E50ADF810504FF40073ADF81230382308
S31508000788ADF81430ADF816500723ADF81830DFF871
S31508000798208202A9404600F057FB2946404600F049
S315080007A887FB0121404600F06FFB3946204600F0DA
S315080007B82BFB4FF40045ADF804508DF806608DF80C
S315080007C8079001A9204600F0CFFA2946204600F0EE
S315080007D81BFB0A27022644463146204600F076FBCC
S315080007E80028F9D0FF21204600F05CFB01252946A0
S315080007F8204600F06BFB0028F9D0013FECD14FF4F6
S315080008080043ADF8043003238DF8063018238DF815
S315080008180730654C01A9204600F0A6FA4FF4805126
S31508000828204600F0F3FA00210846FFF7AFFE012834
S3150800083840F0AE8000F032FF00F57A744FF4D571B7
S315080008480820FFF7A3FE012842D107AE08AF3546B0
S315080008584FF0FF084046FFF74DFE05F8010BBD426D
S31508000868F8D19DF81E30012B40F092809DF81F3074
S31508000878AA2B40F08D804FF08048A92500F00EFF7E
S31508000888844205D941462846FFF780FE0028F5D157
S3150800089800F004FF84427BD900213A20FFF776FE50
S315080008A8002875D1FF242046FFF724FE06F8010B19
S315080008B8BE42F8D19DF81C3003F04003DBB2002B8A
S315080008C814BF0C220422394B1A60FFF73DFE24E0B8
S315080008D80021A920FFF75AFE012887BF01273D46B0
S315080008E80227A925002600F0D9FE844205D93146F3
S315080008F82846FFF74BFE0028F5D100F0CFFE8442C4
S3150800090846D94FF400711020FFF740FE00283FD162
S31508000918264B1F60FFF718FE7FB3224A137803F0A9
S31508000928FE031370224D0021284600F0ADFA002474
S31508000938ADF808404FF48273ADF80A30ADF80C40AC
S31508000948ADF80E40ADF810404FF40073ADF812300C
S315080009580823ADF81430ADF816400723ADF818305B
S3150800096802A9284600F070FA2146284600F0A0FA9F
S315080009780121284600F088FA04E00A4A137843F069
S3150800098801031370074B1878C0B207E001207047B7
S315080009980022064B1A60FFF7D7FDEEE709B0BDE857
S315080009A8F08300BF00000020000C0140440200202C
S315080009B80038004018B9034B1878C0B270470120B0
S315080009C8704700BF00000020002838D170B50D46D2
S315080009D81C46B3B31D4B1B7813F0010F33D11C4BC0
S315080009E81B6813F0080F08BF5202012C0DD11146D7
S315080009F81120FFF7CBFDE0B94FF400712846FFF741
S31508000A083BFEB0FA80F4640913E011461220FFF79A
S31508000A18BDFD70B94FF4007631462846FFF72CFE1F
S31508000A2818B105F50075013CF6D100210C20FFF731
S31508000A38ADFDFFF789FD201C18BF012070BD0420F5
S31508000A487047042070BD032070BD00BF0000002059
S31508000A5844020020002847D170B50D4616461C46A4
S31508000A68002B43D0244B1B7813F0010F40D1224B9F
S31508000A781B7813F0040F3DD1204B1B6813F0080FA1
S31508000A8808BF5602012C0CD131461820FFF77EFD07
S31508000A9820BBFE212846FFF7C1FDB0FA80F4640999
S31508000AA81CE013F0060F03D021469720FFF76EFDCA
S31508000AB831461920FFF76AFD80B9FC2631462846D3
S31508000AC8FFF7ACFD18B105F50075013CF6D1FD2117
S31508000AD80020FFF7A3FD002808BF0124FFF734FD0F
S31508000AE8201C18BF012070BD04207047042070BD63
S31508000AF8032070BD022070BD0000002044020020BB
S31508000B08002840F02681964B1B7813F0010F40F019
S31508000B18228170B584B014460E2900F2FF80DFE8FA
S31508000B2811F00F001500FD005C00FD00FD00FD003A
S31508000B38FD00FD00FD00B700BC00CA00D700E800AC
S31508000B48FFF70EFDB0FA80F46409FEE000210920DB
S31508000B58FFF71CFD002840F0E38010216846FFF7E0
S31508000B688BFD002800F0DE809DF800309B09012BDC
S31508000B7810D19DF808209DF8093003EB02229DF84C
S31508000B8807301B0403F47C13013313449B022360C8
S31508000B980024DAE09DF808209DF807309B0003EB4F
S31508000BA892129DF806309B0203F4406313440133FE
S31508000BB89DF8052002F00F029DF80A1002EBD112E3
S31508000BC8911C9DF80920520002F006020A44D2B286
S31508000BD8093A934023600024B7E0624B1B6813F078
S31508000BE8040F21D000218D20FFF7D0FC002840F003
S31508000BF89B80FF20FFF77EFC10216846FFF73CFD27
S31508000C08002800F093803025FF263046FFF772FC4F
S31508000C186B1E13F0FF05F8D19DF80A301A09102340
S31508000C2893402360002490E000210920FFF7AEFCDA
S31508000C3800287DD110216846FFF71EFD002879D0C7
S31508000C48484B1B6813F0020F11D09DF80A305B0059
S31508000C5803F07E039DF80B2003EBD21301339DF8AE
S31508000C680D209209013A9340236000246DE09DF80F
S31508000C780B10CB0003F0180303EB51119DF80A205B
S31508000C88C2F38402531C01FB0333236000245CE08F
S31508000C98344B1B681370002457E000210920FFF71E
S31508000CA875FC002848D110212046FFF7E5FCB0FA64
S31508000CB880F4640949E000210A20FFF767FCE8BBCD
S31508000CC810212046FFF7D8FCB0FA80F464093CE006
S31508000CD800213A20FFF75AFC90BB651E0334FF260D
S31508000CE83046FFF707FC05F8010FAC42F8D1002497
S31508000CF82BE01C4B1B6813F0040F23D000218D2012
S31508000D08FFF744FC00BBFF20FFF7F4FB4021204611
S31508000D18FFF7B2FCB0FA80F4640916E0042414E07C
S31508000D28012412E0012410E001240EE001240CE05D
S31508000D3801240AE0012408E0012406E0012404E06D
S31508000D48012402E0012400E00124FFF7FDFB204608
S31508000D5803E0042070470320704704B070BD00BF45
S31508000D680000002044020020F0B5CB7803F00F06F7
S31508000D7813F0100F1CBF8B781E430B78F3B1056868
S31508000D88002301274FF00F0C07FA03F20C8832EA02
S31508000D9804040FD19C000CFA04FE25EA0E0506FA8F
S31508000DA804F42543CC78282C01D1426102E0482C6A
S31508000DB808BF02610133082BE6D105600B88FF2BB3
S31508000DC820D94568002301274FF00F0E03F10802C2
S31508000DD807FA02F20C8832EA04040FD19C000EFACC
S31508000DE804FC25EA0C0506FA04F42543CC78282CD5
S31508000DF808BF4261CC78482C08BF02610133082B2A
S31508000E08E4D14560F0BD00BF016170474161704794
S31508000E1821B1054B9A69104398617047024A93694C
S31508000E2823EA0000906170470010024021B1054B83
S31508000E38DA691043D8617047024AD36923EA000081
S31508000E48D06170470010024010B4038803F4415477
S31508000E580A884B8813438A881343CA8813430A891E
S31508000E6813434A8913438A891343CA891343234375
S31508000E789BB20380838B23F400631B041B0C8383B8
S31508000E880B8A038210BC704729B103889BB243F0CA
S31508000E98400303807047038823F040031B041B0C98
S31508000EA80380704781817047808980B2704700BF88
S31508000EB829B103889BB243F400530380704703881B
S31508000EC823F400531B041B0C03807047038919423B
S31508000ED814BF012000207047C1F3080181807047BC
S31508000EE80388194214BF01200020704708B5382125
S31508000EF8014800F097FC08BD14460008F8B5484AAA
S31508000F0802F1240E4FF4FA7748F6A040157854787B
S31508000F182B1903FB077390FBF3F103FB110139B98E
S31508000F2890FBF3F39EB2731E9BB2B3F5806F03D39F
S31508000F3802329645EAD16EE03A4B00225A611A689F
S31508000F4842F400421A601B6813F4004F06D0354F66
S31508000F5800F028FD3B6813F4004FF9D1314B1A68A5
S31508000F6822F002021A601A6842F001021A605B68E7
S31508000F7813F0010F06D12B4F00F014FD7B6813F010
S31508000F88010FF9D0013D013C240544EA0545731EC5
S31508000F981D43244AD561136823F001031360536877
S31508000FA813F0010F06D0144600F0FCFC636813F032
S31508000FB8010FF9D11B4BD3F8002242F00102C3F8FE
S31508000FC80022D3F81C2222F00102C3F81C22D3F807
S31508000FD80C2242F00102C3F80C220022C3F8402270
S31508000FE8C3F84422D3F8042222F00102C3F80422E3
S31508000FF8D3F8142222F00102C3F81422D3F81C22CB
S3150800100842F00102C3F81C22D3F8002222F001029A
S31508001018C3F80022F8BDE421034800F003FC8BE777
S3150800102800470008006400407C46000838B50446B6
S315080010380D46224B9B6813F0806F04D140F22511A8
S315080010481F4800F0EFFB1D4BD3F8802102F0010280
S31508001058C3F88021D3F8802142F07C4242F400127A
S31508001068C3F88021C3F88451E078A1780A0442EAD3
S31508001078006122780A43617842EA0122C3F8882186
S31508001088E079A1790A0442EA006122790A4361797A
S3150800109842EA0122C3F88C21D3F8802142F00102E2
S315080010A8C3F880219B6813F0806F06D1034C00F0C3
S315080010B879FCA36813F0806FF9D038BD0064004046
S315080010C87C4600081F4BDB6813F0030F38D01D4B0E
S315080010D8D3F8B03113F0040F1A4BD3F8B0310EBF5A
S315080010E85B0DDB0843F0004340F26762934220D168
S315080010F8144BD3F8B8210270D3F8B821120A4270F3
S31508001108D3F8B821120C8270D3F8B821120EC2701F
S31508001118D3F8BC210271D3F8BC21120A4271D3F85C
S31508001128BC21120C8271D3F8BC311B0EC371012085
S3150800113800E00020034AD36843F02003D3607047D1
S31508001148002070470064004008B500F067FB08BD3A
S3150800115810B500F06BFA88B100F0E2FB00F08AFAE5
S3150800116800F068FA20F0604020F07F00044B186011
S3150800117800F060FA446800F053FBA04710BD00BFB2
S3150800118808ED00E072B170B50D46561EB6B2441E9B
S31508001198064415F8013B04F8013F00F003FCB44285
S315080011A8F7D170BD704700BF024A136943F0800340
S315080011B8136170470020024070B506460B4D00249F
S315080011C800F0F0FB2B68B3420AD86A6813449E42BB
S315080011D806D204EB4401054B03EB8101087A70BD7E
S315080011E801340C350D2CEBD1FF2070BD24470008BF
S315080011F82DE9F04107460068FFF7DEFFFF2849D0CA
S31508001208264B274A5A6002F188325A603422DA6035
S31508001218DB6813F0010304D0FFF7C6FF0020BDE81A
S31508001228F0811E490A6942F001020A610C463A68C9
S3150800123803EB02081E1DBD59A9B29952E36813F0BB
S31508001248010F05D000F0AEFBE36813F0010FF9D1E2
S315080012582B0CA8F80230E36813F0010F05D000F04C
S31508001268A1FBE36813F0010FF9D1D8F800309D42C5
S3150800127805D13346B6F5007FD9D1012400E000240C
S31508001288064A136923F001031361FFF78DFF204609
S31508001298BDE8F0810020BDE8F08100BF00200240CB
S315080012A82301674538B50D46114B984207D00446C1
S315080012B8104B994208D0FFF79BFF08B911E00E4C6E
S315080012C8C5F308037BB900E0094C2368AB420CD088
S315080012D8204640F8045B4FF400722946FFF752FF90
S315080012E803E0002038BD002038BD204638BD00BFC1
S315080012F848020020006000084C0400202DE9F0414F
S3150800130806460C4617461D4621F4FF7828F00108BC
S315080013180368B3F1FF3F06D140F8048B4FF4007217
S315080013284146FFF72FFF3368984505D041463046B2
S31508001338FFF7B8FF0646E0B13368E41A34440434C4
S3150800134808F5007800F02EFB331DE31AB3F5007F85
S3150800135806D341463046FFF7A5FF064660B1041D89
S3150800136817F8013B04F8013B013DEBD10120BDE824
S31508001378F0810020BDE8F0810020BDE8F08100BFBB
S315080013884FF0FF33024A1360024A1360704700BFE2
S315080013984C0400204802002070B504460D4616463F
S315080013A8FFF70AFFFF2814D0681E2044FFF704FF3A
S315080013B8FF2810D024F4FF7323F00103074A934249
S315080013C82B46324621460CBF05480648FFF796FFC6
S315080013D870BD002070BD002070BD00BF0060000809
S315080013E8480200204C0400202DE9F04106460C4628
S315080013F8FFF7E2FE0546601E3044FFF7DDFE85422C
S3150800140800F286800446EB1EDBB2FB2B00F28380D3
S315080014180F2800F28380434B434A5A6002F1883208
S315080014285A603422DA60DB6813F0010F04D0FFF73C
S31508001438BBFE0020BDE8F0813A4A136943F002036F
S3150800144813613A4FB846002600F0ACFA98F8083007
S31508001458AB4205D106EB4602344B53F8225006E058
S31508001468013608F10C080D2EEED14FF0FF35B846B7
S31508001478002600F097FA98F80830A34205D106EB3B
S3150800148846022A4B53F8228006E0013608F10C0872
S315080014980D2EEED14FF0FF38002600F083FA3B7A7E
S315080014A8A34206D106EB4602204B03EB8202536899
S315080014B804E001360C370D2EEFD10023C5EB0808DA
S315080014C84344C3F38F23CBB15E1EB6B205F58063DA
S315080014D803EB8626134C6561236943F040032361B1
S315080014E8E36813F0010F05D000F05CFAE36813F01F
S315080014F8010FF9D105F58065B542ECD1094A13699A
S3150800150823F002031361FFF74FFE0120BDE8F081BF
S315080015180020BDE8F0810020BDE8F0810020BDE884
S31508001528F08100BF002002402301674524470008D0
S31508001538114B1B68B3F1FF3F18D000B583B00E4BAB
S3150800154859689A681144DA6811441A6911445A693B
S3150800155811449A691144DA698B185B4202AA42F85F
S31508001568043D04210548FFF717FF01E001207047ED
S3150800157803B05DF804FB00BF48020020506100086C
S315080015880D4B1A6804331B6813440C4A1268134433
S315080015980B4A126813440B4A11680B440432126842
S315080015A81A44094B1B681344084A1268D3420CBFED
S315080015B801200020704700BF006000080860000886
S315080015C80C600008106000081860000850610008E0
S315080015D808B50C4B1B68B3F1FF3F04D00948FFF761
S315080015E807FE034660B1084B1B68B3F1FF3F06D0F8
S315080015F80548FFF7FDFD031C18BF012300E001237A
S31508001608184608BD480200204C04002000487047C8
S315080016180060000808B5FFF7B3FE08BD08B5FFF770
S31508001628BBFE08BD08B5FFF7DFFE08BD08B5FFF71E
S31508001638A7FF08BD08B5FFF7E9FF08BD08B5FFF716
S3150800164877FF034610B1FFF7C3FF0346184608BDE0
S31508001658054B00221A60054959609A6005211960E8
S31508001668034B1A60704700BF10E000E03F190100FD
S31508001678500600200022014B1A60704710E000E06F
S31508001688044B1B6813F4803F03D0034A13680133DD
S315080016981360704710E000E05006002008B5FFF711
S315080016A8EFFF014B186808BD500600200E4B1B8833
S315080016B803F080039BB29BB180B20B4B98801B88C2
S315080016C803F080039BB26BB910B5074C00F06AF9B2
S315080016D8238803F080039BB2002BF7D0012010BDA6
S315080016E8002070470120704700440040084B00223C
S315080016F81A819A811A829A821A8340F271221A8169
S315080017089A8992B242F4005242F00C029A817047C2
S3150800171800440040F8B505460C46402903D98D21F2
S31508001728114800F07FF82046FFF7C0FF012803D0CC
S3150800173891210D4800F076F8A3B29BB16C1E013BC7
S315080017489BB21D44084F9A2600F02CF914F8010F8D
S31508001758FFF7ACFF012803D03146384600F062F897
S31508001768AC42F1D1F8BD00BFC047000838B5254BD3
S315080017781C78CCB9244B1B8803F020039BB2002B9A
S315080017883DD0214B9B889BB2204A137013F0FF0368
S3150800179829D0FFF783FF1E4B186000221D4B1A70CD
S315080017A80122184B1A702AE0174B1B8803F02003EE
S315080017B89BB2E3B117490A78134B9D88134B9C18BB
S315080017C865700132D2B20A701B7893420DD112495C
S315080017D8FFF7D8FC00220B4B1A7001240FE00024EF
S315080017E8084B1C700BE01C4609E0002407E0FFF7CD
S315080017F855FF074B1B6864339842F0D800242046E7
S3150800180838BD00BF96060020004400405406002054
S3150800181898060020950600205506002072B67047DF
S3150800182862B6704708B500F0BDF8FCE708B500F0E1
S31508001838B3F8012816D000F0E3FA98B10A4B1B78DA
S31508001848012B0FD1FFF72AFF084B1B6803F5FA731C
S31508001858984207D30022044B1A7000F0D9FA08B93F
S31508001868FFF776FC08BD00BF9C060020A0060020EE
S3150800187808B50122044B1A70FFF710FF034B1860CE
S31508001888FFF7D4FF08BD00BF9C060020A00600206D
S3150800189808B5FFF759FC00F083F8FFF7D9FEFFF7FC
S315080018A8B9FE00F097FA00F00FF8FFF7E1FF08BD58
S315080018B808B500F077F8FFF7E3FE00F0CDFB00F077
S315080018C813F8FFF7B3FF08BD10B500F077F8FFF770
S315080018D815FB044C01232370FFF708FF0023237028
S315080018E810BD00BF0100002008B50B48FFF7EAFB4A
S315080018F8012805D10122094B1A70074800F07CF81F
S315080019080548FFF733FF012805D10022034B1A7053
S31508001918014800F071F808BDA4060020010000205F
S31508001928704700BF38B504460D46084B1B78012B8F
S3150800193802D1C9B2FFF77AFB044B1B781BB9E9B287
S315080019482046FFF7E7FE00F04FF838BD01000020F3
S31508001958074B1B78022B06D0032B06D0012B0CBF8E
S31508001968082040207047002070470020704700BFB5
S3150800197801000020074B1B78022B06D0032B06D044
S31508001988012B0CBF08204020704700207047002014
S31508001998704700BF0100002008B500F01DF808BD13
S315080019A8704700BF704700BF034BFE22DA701871F4
S315080019B80222A3F844207047E4060020054B0022BB
S315080019C81A709A6483F84320A3F844209A705A70C8
S315080019D8704700BFE4060020024B1878003018BF8D
S315080019E801207047E40600200022024B83F84320B2
S315080019F8704700BFE406002038B50378FF2B22D1CC
S31508001A0800F0FEF918B91020FFF7CEFF61E1AD4CDA
S31508001A180023637001252570FF22E27010222271C7
S31508001A286371FFF795FFA071FFF7A4FFE071FFF751
S31508001A38A1FF000A20726572A5720823A4F844302B
S31508001A48FFF7E8FD45E104469E4A1278012A40F068
S31508001A586081C93B352B00F23981DFE813F0C000F5
S31508001A68370137012F01370137012601DB00150138
S31508001A7805013701370137013701370137013701C2
S31508001A883701370137013701370137013701370180
S31508001A983701370137013701370137013701370170
S31508001AA83701370137013701370137013701370160
S31508001AB837017600510036006D00370137013701C6
S31508001AC892003701A400A800B6004578FFF740FF42
S31508001AD80138854203DD2220FFF766FFF9E0794DD4
S31508001AE86278A96C281DFFF74DFBFF23EB70637816
S31508001AF8AA6C1344AB6463780133A5F84430E8E06C
S31508001B084578FFF725FF0138854203DD2220FFF7D0
S31508001B184BFFDEE061686B4DA9646278281DFFF704
S31508001B2831FBFF23EB706378AA6C1344AB646378C4
S31508001B380133A5F84430CCE0624BFF22DA704268DC
S31508001B489A640122A3F84420DDE05E4BFF22DA708E
S31508001B589A6C406840B11044002312F8011B0B44E4
S31508001B68DBB29042F9D100E00023564AC2F80730A2
S31508001B78012313710023537193710823A2F8443083
S31508001B88C1E0504BFF22DA704F4A9A6400221A7154
S31508001B985A719A710721D9711A725A729A72082259
S31508001BA8A3F84420AFE00020FFF7FEFE91E0454B7E
S31508001BB8FF22DA7000221A71597859719A71DA7106
S31508001BC81A720622A3F844209DE03E4B00221A709A
S31508001BD85A70FF22DA700122A3F8442093E0394BA1
S31508001BE89D6CFFF7B5FE621C411E2846FFF716FDD9
S31508001BF818B93120FFF7D8FE6BE0324CFF23E370A3
S31508001C08FFF7A6FE0138A36C0344A3640123A4F8CE
S31508001C18443078E04578FFF79BFE0238854203DDB5
S31508001C282220FFF7C1FE54E0264BFF22DA70012274
S31508001C38A3F84420617839B9FFF700FD002848D190
S31508001C483120FFF7B1FE44E0A21C1E4B986CFFF743
S31508001C58E5FC18B93120FFF7A7FE3AE0194A637878
S31508001C68916C0B44936434E0164CFF23E37000250B
S31508001C7825716571FFF76CFEA071E57125726572AD
S31508001C880723A4F844303EE041680E4B986CFFF7EA
S31508001C98C9FC18B93120FFF787FE1AE0094BFF225D
S31508001CA8DA700122A3F844202DE0FFF751FA054B14
S31508001CB8FF22DA700122A3F8442024E03120FFF736
S31508001CC873FE06E0E4060020444800082020FFF7D3
S31508001CD86BFE104B93F84330012B02D11020FFF707
S31508001CE863FE0C4BB3F94410002912DD0948012399
S31508001CF880F8433089B20330FFF714FE38BD054B28
S31508001D08B3F94410F2E7034B93F84330012BF6D1A5
S31508001D18E4E738BDE406002010B4034602460C483A
S31508001D280131A0FB0242D208FAD100220A70084CF7
S31508001D38A4FB0302D20802EB8200A3EB400330336C
S31508001D4801F8013D1346002AF2D1084610BC70472F
S31508001D58CDCCCCCC70B5441E451C002614F8010F12
S31508001D6802F0D0FBC0B2A0F13003DBB2162B11D8B3
S31508001D78A0F13A02D2B2062A0ED9092B84BFA0F1DD
S31508001D883703DBB203EB061303F0FF06AC42E5D1D3
S31508001D98304670BD002070BD002070BD38B50446B9
S31508001DA80D460009092801D9373003E0303002F01A
S31508001DB8A9FBC0B2287004F00F00092801D93730EA
S31508001DC803E0303002F09EFBC0B268700023AB70A7
S31508001DD8284638BD08B50022054B1A700549064835
S31508001DE801F022FE18B177210448FFF71BFD08BD4C
S31508001DF8700700204C4800087C0700205048000857
S31508001E08024B1878B0FA80F040097047700700202E
S31508001E1808B5FFF7C1FD01280AD0084B1B784BB94E
S31508001E28FEF716FA012807D10122044B1A7008BDD5
S31508001E38002008BD002008BD002008BD7007002046
S31508001E4810B50446007802F05DFB53280DD160787A
S31508001E5802F052FB58B16378312B0AD0322B0AD0DC
S31508001E68332B0CBF0220032010BD032010BD03200E
S31508001E7810BD002010BD012010BD00BF70B5064674
S31508001E880230FFF767FF054684B204363046FFF787
S31508001E9861FF2844C5B2013CA4B20236012CF5D824
S31508001EA83046FFF757FFED43EDB2854214BF0020D1
S31508001EB8012070BD2DE9F04104461646884601B151
S31508001EC820B940F261216348FFF7ACFC2046FFF7CA
S31508001ED8B7FF0546032800F0A0802046FFF7CEFF87
S31508001EE8002800F09D80012D2CD015B1022D5AD05E
S31508001EF89AE0A01CFFF72EFF0746201DFFF72AFFCA
S31508001F080002C8F80000A01DFFF724FFD8F8003023
S31508001F181844C8F800000834F81E07B2002E00F066
S31508001F288680B846002F40F3858000252046FFF7AF
S31508001F3811FF705502340135ADB24545F6DB384612
S31508001F48BDE8F081A01CFFF705FF0746201DFFF72F
S31508001F5801FF0004C8F80000A01DFFF7FBFED8F82B
S31508001F68003003EB0020C8F8000004F10800FFF76A
S31508001F78F1FED8F800301844C8F800000A34381FAB
S31508001F8807B2002E59D0B846002F59DD002520463D
S31508001F98FFF7E0FE705502340135ADB24545F6DB6C
S31508001FA83846BDE8F081A01CFFF7D4FE0746201D79
S31508001FB8FFF7D0FE0006C8F80000A01DFFF7CAFE06
S31508001FC8D8F8003003EB0040C8F8000004F1080010
S31508001FD8FFF7C0FED8F8003003EB0020C8F8000069
S31508001FE804F10A00FFF7B6FED8F800301844C8F816
S31508001FF800000C34781F07B22EB3B846002F25DD2B
S3150800200800252046FFF7A6FE705502340135ADB205
S315080020184545F6DB3846BDE8F0810020BDE8F08185
S315080020284FF0FF30BDE8F0810020BDE8F081384662
S31508002038BDE8F0813846BDE8F0813846BDE8F0814C
S315080020483846BDE8F0813846BDE8F0813846BDE82F
S31508002058F08100BF5048000870B5AC4B1B78002BC0
S3150800206800F0E681012B29D1FFF7D4FAFEF712F919
S31508002078A748FEF753F9A748FEF750F9FEF706F9F9
S3150800208801220146A44801F001FD30B1A348FEF734
S3150800209845F90120FEF736F970BDA148FEF73EF965
S315080020A8A048FEF73BF9A048FEF738F99F4B0022EF
S315080020B81A605A600222954B1A7070BD022B40F0BE
S315080020C8EF809B4C04F50C724FF48071994802F026
S315080020D8F5F894F841326BB19048FEF71FF90220DB
S315080020E8FEF710F904F50C7001F09CFF0022874BE7
S315080020F81A7070BD002874D08E48002200F5C07189
S31508002108FFF7D8FE0446B0F1FF3F0CD18348FEF727
S3150800211805F90320FEF7F6F87F4801F083FF002249
S315080021287A4B1A7070BD00285BDD804B5B6833B943
S315080021387E4B804AD2F880211A60586051E07B4A63
S3150800214812681A447B49D1F88011914203D1034495
S31508002158764A536045E07248FEF7E0F87648FEF797
S31508002168DDF8764E714D31466868FFF7D5FD30467D
S31508002178FEF7D4F87248FEF7D1F83146E878FFF743
S315080021880DFEB11CA878FFF709FE311D6878FFF720
S3150800219805FEB11D2878FFF701FE3046FEF7BEF8A2
S315080021A86848FEF7BBF869682868FFF73BFA60B91C
S315080021B85A48FEF7B3F80520FEF7A4F8564801F082
S315080021C831FF0022514B1A7070BD5548FEF7A6F824
S315080021D85548FEF7A3F8554B564AD2F880211A6097
S315080021E85C60534BD3F84422D3F83C329A4240F009
S315080021F81F810021484801F027FF60B14748FEF7CC
S315080022088DF80420FEF77EF8434801F00BFF0022FC
S315080022183E4B1A7070BD454B5B68002B39D0404859
S31508002228FEF77CF84448FEF779F8444D3F4C2946B2
S315080022386068FFF771FD2846FEF770F84048FEF714
S315080022486DF82946E078FFF7A9FDA91CA078FFF7DD
S31508002258A5FD291D6078FFF7A1FDA91D2078FFF7C0
S315080022689DFD2846FEF75AF83648FEF757F861687E
S315080022782068FFF7D7F960B92848FEF74FF8052010
S31508002288FEF740F8244801F0CDFE00221F4B1A70CD
S3150800229870BD2348FEF742F803221C4B1A7070BD1E
S315080022A8032B40F0C580224C04F50C724FF480715C
S315080022B8204802F003F894F841326BB12248FEF739
S315080022C82DF80220FEF71EF804F50C7001F0AAFE98
S315080022D800220E4B1A7070BD00287CD0154800F5F0
S315080022E8807200F5C071FFF7E5FD0646B0F1FF3FBD
S315080022F82ED11648FEF712F80320FEF703F806480B
S3150800230801F090FE0022014B1A7070BD700700207C
S31508002318C4480008E8480008AC0900201049000825
S31508002328184900082049000844490008740700208D
S315080023387C070020D40B00207449000830070020C9
S3150800234880490008244A00089C490008C049000832
S31508002358002840DD3748FDF7E1FF374C214630466F
S31508002368FFF7DAFC2046FDF7D9FF3448FDF7D6FF14
S31508002378334D214695F88301FFF710FDA11C95F802
S315080023888201FFF70BFD211D95F88101FFF706FD70
S31508002398A11D95F88001FFF701FD2046FDF7BEFF50
S315080023A82848FDF7BBFF05F580723146D5F8800148
S315080023B8FFF734F960B92448FDF7B0FF0620FDF7A2
S315080023C8A1FF224801F02EFE0022214B1A7070BD8B
S315080023D82048FDF7A3FF204BD3F84422D3F83C3214
S315080023E89A4225D11D48FDF799FFFFF727F960B9E5
S315080023F81548FDF793FF0720FDF784FF134801F0FA
S3150800240811FE0022124B1A7070BD1248FDF786FF9E
S315080024181348FDF783FF0D4801F004FE1148FDF740
S315080024287DFF00220A4B1A70FDF748FFFEF790FE5B
S3150800243870BD00BFE449000830070020F4490008C9
S31508002448D40B0020244A000810490008AC090020CB
S3150800245870070020184900087C0700200C4A000865
S31508002468284A0008404A0008C278837843EA0222C4
S31508002478437843EA0223007840EA0320704700BFFE
S315080024883AB101388A1811F8013B00F8013F914220
S31508002498F9D1704702394369023B99423DBF4389DE
S315080024A8806A01FB03000020704700BF00F10B019A
S315080024B80023DA0142EA530310F8012B134403F008
S315080024C8FF038842F5D11846704700BF0168E1B195
S315080024D810B40C781F2C09D93A2C1FD00A4612F8C2
S315080024E8013F1F2B04D93A2BF9D105E023460A46A2
S315080024F83A2B18BF002013D14B1C9A4208D1302C0E
S3150800250809D10231016000200AE04FF0FF30704718
S315080025184FF0FF3004E04FF0FF3001E00A46EBE7E2
S3150800252810BC704738B50C4670B1054603685BB1F0
S315080025381A784AB1D9888288914205D15878FEF71F
S3150800254839FA10F0010F03D000232360092038BD9B
S315080025582B682360002038BDC37833B32DE9F041D2
S315080025680446C56A00F1300701232A4639464078E9
S31508002578FEF770FAD8B90023E370236AEB1AA26942
S31508002588934217D2A678012E17D94FF00108A369E6
S315080025981D4443462A4639466078FEF75BFA013EEB
S315080025A8012EF4D10020BDE8F081002070470120F3
S315080025B8BDE8F0810020BDE8F0810020BDE8F08183
S315080025C870B5C36A8B4213D004460D46FFF7C4FF9D
S315080025D8064670B901232A4604F130016078FEF7E9
S315080025E8F3F900281CBF01264FF0FF35E56200E025
S315080025F80026304670BD00BF10B50446FFF7ACFF8D
S315080026080346002852D12378032B47D12379012B77
S3150800261844D104F1300104F50C700B46002203F886
S31508002628012B8342FBD1552384F82E32AA2384F83A
S315080026382F32522384F8303084F83130612384F8F5
S315080026483230412284F83320722084F8140284F840
S31508002658150284F8162284F81732236984F8183282
S315080026681A0A84F819221A0C84F81A221B0E84F8F6
S315080026781B32E36884F81C321A0A84F81D221A0CDD
S3150800268884F81E221B0E84F81F32E2690132E262C0
S3150800269801236078FEF7DEF900232371002211462C
S315080026A86078FEF72DFA031C18BF0123184610BDDB
S315080026B82DE9F843012940F283804369994280F05D
S315080026C8818017460C4605460378022B3DD0032B16
S315080026D851D0012B78D101EB5108016A01EB582139
S315080026E8FFF76EFF0646002840F0858008F10109C5
S315080026F8C8F3080814F0010F13D0A84498F8303026
S3150800270803F00F0343EA071388F830300123EB7008
S31508002718296A01EB59212846FFF752FF002859D0A4
S3150800272854E0A84488F830700123EB70296A01EB55
S3150800273859212846FFF744FF002850D048E0A94405
S3150800274889F830200123EB7055E0016A01EB142162
S31508002758FFF736FF064600284DD1630003F4FF73DA
S31508002768EA1882F830701346C7F3072283F831202F
S315080027780123EB703FE0016A01EBD411FFF720FF54
S315080027880646C0BB27F07047A40004F4FE7404F19B
S315080027983008A8444046FFF767FE00F0704040EA54
S315080027A807022C4484F83020130A88F80130130CE1
S315080027B888F80230120E88F803200123EB701AE015
S315080027C8022618E0022616E0022614E0064612E05B
S315080027D8064610E0C9F30809C7F30712AFE7C9F3B5
S315080027E8080905EB090393F8303023F00F03C7F3FC
S315080027F803221A43A3E73046BDE8F8838A76C2F36C
S315080028080723CB760378032B03D1120C0A75120A11
S315080028184A7570472DE9F84300238B758369002BA1
S3150800282872D00D460646436AB3F1FF3F1DD0836A48
S315080028389F1C188888B101F115080024A146494645
S3150800284801F092FD58B1FF2C0BD0013408F8010F9E
S3150800285837F8020B0028F2D104E0002402E000242D
S3150800286800E000242C440023A375A87D00242346F1
S315080028782E275A1CF169CB5C202B22D0052B08BFC2
S31508002888E523092A05D108B929198F7529194F7217
S31508002898013429194B7298B9A3F14101C9B219290A
S315080028A80CD8F169097B082A8CBF4FF0100E4FF037
S315080028B8080E1EEA010F1CBF2033DBB229198B75D7
S315080028C8013413460B2AD4D138B92B1900229A7524
S315080028D8F3691B7B934208BF14462C440023637292
S315080028E8F369DB7A2B72F0691C30FFF7BDFD2860A7
S315080028F8F269517E137E43EA0123AB80F269D17DE2
S31508002908937D43EA0123EB80BDE8F883012955D96D
S31508002918F8B506687369994252D20C463378022B81
S3150800292829D0032B39D0012B4CD101EB5105316A3B
S3150800293801EB55213046FFF743FE002844D16F1CAA
S31508002948C5F30805354495F83050316A01EB572127
S315080029583046FFF735FE002839D1C7F308073E4445
S3150800296896F8300045EA002014F0010F14BF000954
S31508002978C0F30B00F8BD316A01EB14213046FFF7A6
S315080029881FFE38BB610001F4FF71731893F8310014
S3150800299893F8303043EA0020F8BD316A01EBD411C8
S315080029A83046FFF70DFEC0B9A00000F4FE703030BF
S315080029B83044FFF759FD20F07040F8BD01207047F4
S315080029C80120F8BD0120F8BD4FF0FF30F8BD4FF0E3
S315080029D8FF30F8BD4FF0FF30F8BD4FF0FF30F8BDB7
S315080029E8B1F5001F46D22DE9F04106460C4611F00E
S315080029F81F0F41D1D0F800803161856885B998F8EC
S31508002A080030022B02D9D8F8243043B9B8F8083070
S31508002A18B3EB541F33D9D8F82430B3611BE01D46ED
S31508002A28B8F80A707F02BC4210D329463046FFF729
S31508002A386DFF0546B0F1FF3F24D0012825D9D8F8FF
S31508002A481430984224D2E41BA742EED929464046B8
S31508002A58FFF720FDB0617561B369E3B103EB542351
S31508002A68B36108F13003C4F308042344F361002072
S31508002A78BDE8F081022070470220BDE8F0810220F7
S31508002A88BDE8F0810120BDE8F0810220BDE8F081AB
S31508002A980220BDE8F0810220BDE8F0812DE9F04169
S31508002AA807460668884631B9F56885B173699D424F
S31508002AB828BF01250CE0FFF729FF012846D9B0F100
S31508002AC8FF3F46D07369984252D3454600E0012530
S31508002AD82C46013473699C4202D3012D3DD9022440
S31508002AE821463846FFF712FF38B1012838D0B0F129
S31508002AF8FF3F38D0AC42ECD139E04FF0FF322146DF
S31508002B083046FFF7D5FD0346C8B9B8F1000F06D019
S31508002B18224641463046FFF7CBFD034678B9F460AE
S31508002B2833697269023A93423CBF03F1FF33336152
S31508002B38337943F0010333712046BDE8F081012B50
S31508002B480CBF4FF0FF300120BDE8F0810120BDE839
S31508002B58F0814FF0FF30BDE8F0810020BDE8F08134
S31508002B680120BDE8F0814FF0FF30BDE8F081002074
S31508002B78BDE8F0812DE9F0410E46012930D907460E
S31508002B881146046863699E422DD22AB14FF0FF3276
S31508002B982046FFF78DFD48BB4FF0000831463846FA
S31508002BA8FFF7B4FE054618B3012824D0B0F1FF3F55
S31508002BB824D0424631462046FFF77AFD08BB2369EA
S31508002BC8B3F1FF3F05D001332361237943F00103AD
S31508002BD823712E4663699D42E0D30020BDE8F08143
S31508002BE80220BDE8F0810220BDE8F081BDE8F08149
S31508002BF80020BDE8F0810220BDE8F0810120BDE88B
S31508002C08F081BDE8F08100BF8369002B76D02DE9F5
S31508002C18F04705692035B5F5001F71D28846044680
S31508002C280668C5F30807002F61D101338361416936
S31508002C3841B93389B3EB551F59D80023836104205A
S31508002C48BDE8F0877389013B13EA55234FD1FFF78F
S31508002C585DFE8146012856D9B0F1FF3F56D0736903
S31508002C6898423DD3B8F1000F04D10023A36104208C
S31508002C78BDE8F08761692046FFF710FF81460028FE
S31508002C8847D0012848D0B0F1FF3F48D03046FFF773
S31508002C9863FC002846D106F1300306F50C710022BC
S31508002CA803F8012B8B42FBD149463046FFF7F2FB66
S31508002CB8F0624FF000084FF0010A0AE086F803A010
S31508002CC83046FFF749FC80BB08F10108F36A01336F
S31508002CD8F36273899845F1D3F36AC8EB0303F36281
S31508002CE8C4F8149049463046FFF7D4FBA06125611D
S31508002CF830373744E7610020BDE8F087042070477D
S31508002D080420BDE8F0870220BDE8F0870120BDE869
S31508002D18F0870720BDE8F0870220BDE8F087012084
S31508002D28BDE8F0870120BDE8F0870120BDE8F087F7
S31508002D382DE9F843044605680669416AB1F1FF3F7B
S31508002D4803D0FFF74DFE0346D8B94FF0E50801272B
S31508002D584FF00009A1692846FFF732FC034668B90F
S31508002D68E26982F80080EF702269964209D94946D5
S31508002D782046FFF749FF03460028EBD0042B08BF77
S31508002D8802231846BDE8F8832DE9F04F85B00546B5
S31508002D98D0F800B00021FFF723FE002840F0A680EF
S31508002DA84FF0FF336B624FF0FF0AD1461F46A969F9
S31508002DB85846FFF705FC002840F09980EC69267804
S31508002DC8002E00F09580E37A03F03F02AA71E52EFB
S31508002DD804D013F0080F05D00F2A05D06F624FF0FC
S31508002DE8FF097BE00F2A5AD1D5F82880B8F1000FD9
S31508002DF874D016F0400F06D094F80DA006F0BF065A
S31508002E082B696B6204E0B14518BF4FF0FF0965D11D
S31508002E18637B009353455FD1E27EA37E53EA022380
S31508002E287DD1237803F03F03013B03EB430203EB11
S31508002E388203DFF80CA10121CDF804B003961E46DB
S31508002E4802951AF8013BE2185578E35C43EA05252A
S31508002E5881B1FE2E58D8284601F0A8FA834606F10D
S31508002E68010938F8160001F0A1FA834550D1294618
S31508002E784E4603E04FF6FF739D424DD12F4B5345FF
S31508002E88DFD1DDF804B03246039E029D237813F09D
S31508002E98400F33D091B338F812307BB33FE0B9F11D
S31508002EA8000F04D12046FFF701FB824522D02A6A83
S31508002EB8D37A13F0010F37D00AE011F8013B10F85E
S31508002EC8012B9B1A8C4202D0002BF6D000E09BB14E
S31508002ED86F624FF0FF0901E04FF0FF09002128460D
S31508002EE8FFF792FE00283FF462AF24E023E022E0D1
S31508002EF8042020E000201EE000201CE0013E5FFAC6
S31508002F0886F9DDF800A0E9E7DDF804B0029D06E0D9
S31508002F18DDF804B0029D02E0DDF804B0029DDDF894
S31508002F2800A04FF0FF09D9E7611C501C14F80B3BA9
S31508002F3812789B1AC8E705B0BDE8F08F0D4B000854
S31508002F48004B00082DE9F04F8BB0076AFB7A13F09F
S31508002F58A00F40F03E81D0F828A0BAF800304BB14F
S31508002F6853464FF0000808F1010833F8022F002AE3
S31508002F78F9D101E04FF000080446036801930C22D2
S31508002F88394607A8FFF77CFA9DF8273013F0010F92
S31508002F9875D00023FB72A3620B2207A93846FFF7F0
S31508002FA86FFA012633464FF07E0920251FE00B22CB
S31508002FB807A93846FFF764FA052E17D9AAF1020EAB
S31508002FC833460EE0102102F0010000EB43035208D5
S31508002FD813F4803F1CBF83F4883383F02103013937
S31508002FE8F1D13EF8022F002AECD100E033460DF164
S31508002FF81C0E072203F00F0000F13001392988BF9B
S3150800300800F13701013A0EF8011D1B09F2D10AAB86
S31508003018134403F8149C62B13B78202B0BD039462D
S31508003028002301339A4207D011F8010F2028F8D156
S3150800303802E0002300E00023F9180133072A05D81F
S315080030480AA8104410F8140C013200E0284601F8C2
S31508003058010B072BF1D92046FFF796FE20B9013652
S31508003068642EA4D10720D3E0642E00F0B480042887
S3150800307840F0B3809DF82730FB72C4F828A09DF865
S31508003088273013F0020F07D008F10C08624DA5FB8C
S315080030980835AD08013500E00125276800212046D6
S315080030A8FFF79EFC0346002840F0AC8000264FF048
S315080030B80108A1693846FFF783FA0346002840F055
S315080030C8A180E3691B78E52B00D01BB90136B54208
S315080030D801D19AE0002641462046FFF795FD0346AA
S315080030E80028E6D08EE02169A1EB45112046FFF7B6
S315080030F877FC034600287CD1206AFFF7D7F90290A7
S3150800310800260396A1690198FFF75AFA034600288C
S315080031186FD1D4F82880E1695FFA85F99DF80830F7
S315080031284B734FF00F03CB720E738E76CE7609F17A
S31508003138FF3303EB430003EB8000384A02F10D0C1A
S31508003148039B4FF6FF774FF0FF0ABB4248D000F1C2
S31508003158010E38F81030107801EB000B0B54180ADA
S315080031688BF8010013B970463B4600E070460132F9
S315080031786245EAD14FF6FF72934202D038F810300A
S315080031880BB949F0400981F800900123019AD370D8
S3150800319831462046FFF738FD034650BB013DB1D1FD
S315080031A829E0E36903F12001002203F8012B99427B
S315080031B8FBD10B22216AE069FFF762F9E269236A03
S315080031C8DB7A03F0180313730123019AD3700020DE
S315080031D81EE006201CE007201AE019E0072017E081
S315080031E892F800E001EB0E0B01F80EA08BF801A08F
S315080031F8BDE718460CE0A1690198FFF7E1F9002830
S31508003208CFD005E0042BE9D0F3E7013DF3D06AE710
S315080032180BB0BDE8F08F00BF4FECC44E004B00085A
S3150800322810B504460023C3704FF0FF33C362FFF797
S31508003238C7F9F0B994F82F2294F82E3243EA0223F4
S315080032481BB20F4A934216D104F16600FFF70CF930
S3150800325820F07F400B4B98420FD004F18200FFF70D
S3150800326803F920F07F40074B984214BF022000203C
S3150800327810BD042010BD032010BD002010BD00BFDE
S3150800328855AAFFFF464154002DE9F04385B00E467E
S31508003298174600230B60FFF719F9051EC0F22E81A1
S315080032A8C04B53F82540002C00F02A81346007F0FB
S315080032B8FE07237883B16078FDF77CFB10F0010FD1
S315080032C80AD1002F00F01E8100F00400C0B20028C1
S315080032D80CBF00200A206FE100232370E8B2607053
S315080032E8FDF7F8F910F0010F40F00E811FB110F044
S315080032F8040F40F00B8100212046FFF791FF0228B2
S3150800330825D16E4604F5FB7504F236286F464FF04C
S31508003318000915F8043C1BB12846FFF7A5F800E094
S31508003328484647F8040B1035A845F2D104AF4FF0C4
S31508003338030856F8045B35B129462046FFF770FF9F
S31508003348012801D802E14046BE42F2D100E0002534
S31508003358042800F0DD80012888BF0D2000F22C81A2
S3150800336894F83C2094F83B3043EA02231BB2B3F5A1
S31508003378007F40F0CF8094F8477094F8463053EAB7
S31508003388072704D104F15400FFF76EF80746A7612A
S3150800339894F8409084F8029009F1FF33DBB2012BC8
S315080033A800F2BA8094F83D60B3B26381002B00F04E
S315080033B8B580731E334240F0B38094F8428094F87F
S315080033C8413043EA0828A4F8088018F00F0F40F09F
S315080033D8A98094F8440094F8433053EA002003D1AE
S315080033E804F15000FFF740F894F83F2094F83E306F
S315080033F853EA022300F0988007FB09F903EB181132
S3150800340849448842C0F09280401AB0FBF6F6002E6E
S3150800341800F08E8040F6F572964294BF0122022289
S315080034284FF6F570864200F2958002366661E561C8
S315080034382B4423622944A162032A15D194F85B20F8
S3150800344894F85A3053EA022374D1B8F1000F73D1AD
S3150800345804F15C00FFF708F86062B30003F2FF1393
S31508003468B7EB532F6AD38AE0B8F1000F68D04B44FC
S315080034786362022A0FBF760006EB460306F00106CA
S3150800348806EB530675E0691C2046FFF799F828BB32
S315080034980023237194F82F2294F82E3243EA022344
S315080034A81BB2414A93421BD104F13000FEF7DCFFF8
S315080034B83E4B984216D104F50570FEF7D5FF3C4BEE
S315080034C8984211D104F50670FEF7CEFF206104F57F
S315080034D80770FEF7C9FFE060032206E0032204E04E
S315080034E8032202E0032200E003222270314A1388ED
S315080034F801339BB21380E38000205DE00B205BE07C
S315080035080C2059E0002057E0032055E00A2053E034
S31508003518012051E00D204FE00D204DE00D204BE035
S315080035280D2049E00D2047E00D2045E00D2043E039
S315080035380D2041E00D203FE00D203DE00D203BE049
S315080035480D2039E0012037E00D2035E004287FF406
S3150800355807AFF7E702366661E5612B4423626B1805
S31508003568A3626BE74FF0FF332361E360802323717F
S31508003578BBE706F2FF16B7EB562FE5D3F2E74FF08F
S31508003588FF332361E3608023237194F8612094F85C
S31508003598603043EA02231BB2012B3FF474AF0322BF
S315080035A8A3E700BF5C0F002055AAFFFF52526141EE
S315080035B872724161580F002005B0BDE8F08300BF5C
S315080035C82DE9F04F83B00446894607684FF0FF0A8D
S315080035D855460426D0464FF6FF7B7AE03846FEF76E
S315080035E8EFFF0646002878D1E0690378002B7ED0DD
S315080035F8C27A02F03F02A271E52B5DD02E2B5DD070
S3150800360822F02001082914BF00210121494557D174
S315080036180F2A48D113F0400F06D090F80DA003F0F2
S31508003628BF032269626203E09D4218BF45464AD134
S3150800363890F80DE0D64545D1C17E827E52EA012230
S315080036484ED1A26A11460192027802F03F02013A67
S3150800365802EB420602EB8606284D05F10D0A4FF0E5
S31508003668010C009363468C4615F8012B8118497896
S31508003678825C42EA012233B1FE2E31D82CF8162094
S315080036881346013601E05A452AD1AA45ECD1009BD2
S31508003698027812F0400F26D0FE2E21D80022019972
S315080036A821F816201FE01DB9FEF700FF824520D035
S315080036B84FF0FF3363621CE0454604E0454602E0E6
S315080036C8454600E0454600212046FFF79DFA06468E
S315080036D818B9A169002981D15EB10023A36108E060
S315080036E8F2464546EFE7013BDDB2F246EBE704262C
S315080036F8F3E7304603B0BDE8F08F00BF004B00087B
S31508003708CA7E8B7E43EA02230278032A05D1487DBE
S315080037180A7D42EA002243EA02431846704700BF78
S315080037282DE9F04F85B00546D0F80090884611F87F
S31508003738013B2F2BFAD05C2BF8D00023AB6098F806
S3150800374800301F2B08D82B6A8022DA7200212846F7
S31508003758FFF746F903465CE14FF0010AAE6A98F8A6
S3150800376800001F280DD92F280ED05C280FD0A6F1E7
S31508003778020B474601241AE02F280AD05C2811D1E3
S3150800378807E00024534604E00024534601E00024D9
S3150800379853464344984613F8012B2F2AFAD05C2A35
S315080037A8F8D01FE0B3F5807F00F029811C46514602
S315080037B800F0DAFD0146002800F021817F2809D8A3
S315080037C8222800F0E880954A12F8013F13B198427A
S315080037D8FAD1E0E02BF8021F631C17F8010F1F281F
S315080037E8CAD8D6E7202834BF04270027002C00F0BB
S315080037F8F28006EB440232F8023D202B01D02E2B2C
S3150800380803D1013CF7D1B346E6E06000002326F869
S315080038181430002C00F0F3802B6A03F10B012022E8
S3150800382803F8012B9942FBD1B11E002300E00133AE
S3150800383831F8022F202AFAD02E2AF8D0002B00F0C9
S31508003848CF8047F00307CBE0013C05D10822019257
S3150800385800220292039204E032F8021D2E29F3D1BF
S31508003868F4E703F1010B36F81300002860D0202886
S3150800387803D02E2805D1A34503D047F003075B4696
S31508003888EFE7029B019A934202D2A34519D1B8E001
S31508003898019B0B2B06D147F003072B6A1A78E52AF2
S315080038A856D14AE0A34502D047F0030740D8039B00
S315080038B89B00DBB2039323460B220192082202924D
S315080038C8CFE77F2840F29380002100F04DFD03469C
S315080038D8002800F09B80524A134413F8801C88B2CB
S315080038E847F0020740B12B2906D04E4A12F8013F85
S315080038F8002B7ED08B42F9D147F003075F200FE0F3
S31508003908039B43F0020303930AE0A0F161039BB209
S31508003918192B05D8039B43F001030393203880B27B
S315080039282B6A02990A4658545B460132029298E76E
S315080039382B6A1A78E52A04D101E00B22019205229E
S315080039481A70019B082B03D1039B9B00DBB20393D8
S31508003958039A02F00C030C2B03D002F00302032A85
S3150800396801D147F0020717F0020F0AD1039A02F0AD
S315080039780302012A08BF47F01007042B08BF47F0BF
S3150800398808072B6ADF722846FFF7FEF92B6ADA7AE8
S31508003998034660B101E006233BE0042839D102F06A
S315080039A80402D2B2002A14BF0346052331E012F0F6
S315080039B8040F2ED1AB7913F0100F0AD02B69C3F375
S315080039C8080303F1300149444846FFF799FEA86001
S315080039D8C4E605231DE0B3460023ABF80030DAE752
S315080039E802383218315A2E293FF430AF2CE70146EF
S315080039F879E7A0F141039BB2192B81D985E70623FC
S31508003A0807E0019B0B2B7FF452AF44E747F0020708
S31508003A1872E7184605B0BDE8F08F00BF6C4A000883
S31508003A28804A0008784A000810B584B001900091C9
S31508003A38144604A840F8041DFEF748FD002816DBBE
S31508003A48114B53F820300BB100221A70019BA3B111
S31508003A5800221A70019B0C4A42F820304BB1012CFF
S31508003A6809D1002201A96846FFF70EFC0AE00B20D7
S31508003A7808E0002006E0002004E00023024A42F895
S31508003A882030184604B010BD5C0F00202DE9F0431D
S31508003A9893B00191002800F09C800446154600233F
S31508003AA8036002F01F06324606A901A8FFF7ECFBD9
S31508003AB8002840F09080069B079303AB0F935A4B58
S31508003AC81193019907A8FFF72BFE0346002840F033
S31508003AD883800F9B93F90B30002B80F288807FE058
S31508003AE8042B40F08C8007A8FFF72CFA46F0080646
S31508003AF8034650B193E09DF8223013F0110F40F0B9
S31508003B08878015F0040F40F0858016F0080F46D018
S31508003B180E9B00259D73DD736121197448225A741A
S31508003B280E9B9D75DD7519765A7620220E9BDA72DC
S31508003B38069FDDF8388041463846FFF7E1FD81469D
S31508003B482A4641463846FEF759FE0E9B1D775D778D
S31508003B589D77DD770122069BDA70B9F1000F1CD034
S31508003B68069BDD6A0022494607A8FFF703F80346BD
S31508003B78002854D129460698FEF722FD09F1FF3395
S31508003B88069AD36048B14BE015F0020F02D013F03D
S31508003B98010F41D115F0080F01D046F02006069B03
S31508003BA8DB6A23620E9B6362069D0E9F394628468A
S31508003BB8FFF7A6FDA06007F11C00FEF755FCE060BC
S31508003BC8002060746061E06126742560EB88A38034
S31508003BD826E0092024E023E015F01C0F0BD07FE728
S31508003BE815F01C0F18BF062309D1062303E015F0A4
S31508003BF81C0F80D106E0002BD6D0184610E046F0F8
S31508003C080806F8E79DF8223013F0100F06D1BBE72F
S31508003C18072005E0082003E0072300E004231846E8
S31508003C2813B0BDE8F08300BF580D00202DE9F04F0A
S31508003C3885B00446884615461F4600233B6003A9F7
S31508003C48FEF770FC002840F0A280607C002840F04F
S31508003C58A280237C13F0010F00F09A80E368666956
S31508003C689E1BAE4228BF2E46002E00F0938004F114
S31508003C78280301936369C3F30802002A6DD1039ADE
S31508003C885289013A12EA532912D10BB9A06803E0FE
S31508003C98A1692046FEF73AFE012802D80220607478
S31508003CA879E0B0F1FF3F02D10120607473E0A061AA
S31508003CB8DDF80CA0A1695046FEF7ECFB054610B9DD
S31508003CC80220607467E04D445FEA562B24D0BAF8A0
S31508003CD80A3009EB0B029A4288BFC9EB030B5B460D
S31508003CE82A4641469AF80100FCF76EFE10B10120F3
S31508003CF8607450E0237C13F0400F0AD0E069401B3B
S31508003D08834506D94FF40072019908EB4020FEF75F
S31508003D18B7FB4FEA4B252EE0E26995421CD0237C77
S31508003D2813F0400F0DD0012301999AF80100FCF70A
S31508003D3891FE10B1012060742DE0237C23F0400326
S31508003D48237401232A46019903984078FCF73CFE18
S31508003D5810B1012060741EE0E5616169C1F30801CC
S31508003D68C1F50075B54228BF354628312A4621448B
S31508003D784046FEF785FBA84463692B4463613B68A4
S31508003D882B443B60761B7FF475AF002003E002E006
S31508003D98072000E0002005B0BDE8F08F2DE9F04FB8
S31508003DA885B00446884616461F4600233B6003A985
S31508003DB8FEF7B8FB002840F0BD80607C002840F07C
S31508003DC8BB80237C13F0020F00F0B5806369F342C9
S31508003DD828BFDE43002E00F0A78004F128030193CC
S31508003DE86369C3F30802002A7DD1039A5289013A06
S31508003DF812EA53291DD133B9A06858B900212046BB
S31508003E08FEF74CFE03E0A1692046FEF747FE0028A8
S31508003E1800F08A80012802D1022060748CE0B0F193
S31508003E28FF3F02D10120607486E0A061A36803B948
S31508003E38A060237C13F0400F0ED00123E269019994
S31508003E4803984078FCF706FE10B10120607473E009
S31508003E58237C23F040032374DDF80CA0A16950469F
S31508003E68FEF718FB054610B90220607464E04D4455
S31508003E785FEA562B24D0BAF80A3009EB0B029A42A5
S31508003E8888BFC9EB030B5B462A4641469AF80100E8
S31508003E98FCF7E0FD10B1012060744DE0E169491BAB
S31508003EA88B450AD94FF4007208EB41210198FEF7B1
S31508003EB8E7FA237C23F0400323744FEA4B2524E0D2
S31508003EC8E3699D420ED06269E3689A420AD20123E1
S31508003ED82A4601999AF80100FCF776FD10B10120E7
S31508003EE8607429E0E5616069C0F30800C0F50075EB
S31508003EF8B54228BF354628302A4641462044FEF7AB
S31508003F08BFFA237C43F040032374A84463692B440F
S31508003F186361E268934238BF1346E3603B682B4403
S31508003F283B60761B7FF45CAF237C43F02003237445
S31508003F38002001E000E0072005B0BDE8F08F00BFCB
S31508003F4870B582B004460E460A2902D10D21FFF73C
S31508003F58F7FF6368002B14DB5D1C23441E733C2D96
S31508003F680BDD01AB2A4604F10C012068FFF716FFA2
S31508003F78019B5D1B18BF4FF0FF356560A3680133C9
S31508003F88A36002B070BD00BF30B583B0044601A96E
S31508003F98FEF7C8FA00283ED1237C13F0200F3BD041
S31508003FA813F0400F0CD00123E26904F128010198A7
S31508003FB84078FCF74FFD88BB237C23F04003237425
S31508003FC8216A0198FEF7FCFA50BB656AEB7A43F05A
S31508003FD82003EB72A26829462068FEF70FFCE368FF
S31508003FE82B771A0A6A771A0CAA771B0EEB7700231F
S31508003FF8AB75EB7561222A7648226A76AB74EB7440
S315080040080122019BDA700198FEF7F6FA237C23F061
S315080040182003237404E003E0002001E00120FFE701
S3150800402803B030BD10B582B00446FFF7ADFF0346AE
S3150800403838B901A92046FEF775FA034608B90022D9
S315080040482260184602B010BD70B582B004460D4607
S3150800405801A9FEF767FA002840F0A880607C0028C6
S3150800406840F0A880E268AA4206D2237C03F002033D
S31508004078DBB2002B08BF1546636900226261002D72
S3150800408800F09580019A568976026BB1013B6A1E43
S31508004098B2FBF6F2B3FBF6F18A4205D37242134035
S315080040A86361ED1AA16912E0A16879B92046FEF79D
S315080040B8F5FC0146012802D1022060747AE0B0F1C5
S315080040C8FF3F02D10120607474E0A060A161002955
S315080040D837D0B54225D9237C13F0020F05D02046E0
S315080040E8FEF7DCFC014620B91AE02046FEF70EFC6E
S315080040F80146B1F1FF3F02D1012060745AE0012957
S3150800410803D9019B5B69994202D30220607451E086
S31508004118A161636933446361AD1BAE42DBD300E03A
S31508004128354663692B446361C5F308035BB1019897
S31508004138FEF7B0F910B9022060743BE000EB55258C
S3150800414802E0002500E000256369C3F3080313B3FA
S31508004158E26995421FD0237C13F0400F0ED0012345
S3150800416804F1280101984078FCF774FC10B1012085
S3150800417860741FE0237C23F04003237401232A4636
S3150800418804F1280101984078FCF71EFC10B10120BB
S3150800419860740FE0E5616369E268934209D9E360F0
S315080041A8237C43F020032374002003E002E0002068
S315080041B800E0002002B070BD30B591B001900D4600
S315080041C8002205A901A8FFF75FF80446A8B902ABBB
S315080041D80D930B4B0F93019905A8FFF7A1FA04460F
S315080041E858B90D9B93F90B30002B05DB2DB12946E1
S315080041F805A8FEF70FFB00E00624204611B030BDDF
S31508004208580D002070B59CB00190022205A901A896
S31508004218FFF73AF8059B11930346002848D102ABE5
S315080042281993254B1B93019911A8FFF779FA0346A9
S3150800423800283DD1199B93F90B30002B35DB9DF8E7
S315080042484A4014F0010F32D11DE006950896002160
S3150800425806A8FEF7C5FB034650BB002106A8FFF7CC
S31508004268AFF90346F8B1042816D021E036B1002282
S31508004278314611A8FEF77EFC0346C8B90598FEF72D
S31508004288BBF9034614E0059D18992846FFF738FA3E
S31508004298064614F0100FD8D111A8FEF749FD0346B3
S315080042A80028E3D004E0072302E0062300E00723FA
S315080042B818461CB070BD00BF580D00202DE9F04106
S315080042C882B080461746054600244E1E12E06B4605
S315080042D8012201A93846FFF7A9FC009B012B0DD13D
S315080042E89DF804300D2B05D06A1C2B7001340A2B57
S315080042F803D01546B442EADB00E0154600232B70C6
S315080043089C4214BF4046184602B0BDE8F08100BF7B
S3150800431810B594B0044601910023029303930178DB
S3150800432851B101A8FFF70CFE14F8011F0029F8D1AE
S31508004338029A002A01DA0CE000226B4604A90198C1
S31508004348FFF72CFD40B9009B029A9A4207D10398B9
S3150800435807E04FF0FF3004E04FF0FF3001E04FF080
S31508004368FF3014B010BD00BF7F281BD911B9C72864
S3150800437808D112E0FF2814D8A0F180030A4A32F8B7
S3150800438813007047084A012332F8021F814205D0F4
S3150800439801339BB2802BF7D100E000238033D8B2D3
S315080043A870470020704700BF104B0008F0B5244935
S315080043B8244BB0F5805F38BF1946074604310C46CA
S315080043C831F8043C002B39D0984237D331F8022CFF
S315080043D8150AD2B2BE46D618B04229DA082D2DD803
S315080043E8DFE805F0050A101316191C1F2200C3EB8F
S315080043F8070E31F81E00F0BDC31A03F00103C01AF0
S3150800440880B2F0BD103880B2F0BD203880B2F0BD59
S31508004418303880B2F0BD1A3880B2F0BD083080B2A4
S31508004428F0BD503880B2F0BDA0F5E35080B2F0BDBB
S315080044380431002DC3D104EB4201BFE7F0BD00BF2C
S31508004448104C0008CC4C00087F2805D8034B185C8C
S31508004458034B5B5C184070470020704758510008AA
S31508004468EC4F0008A0F16103192B98BF2038704754
S31508004478A0F14103192B98BF203070477F2805D82B
S31508004488034B185C034B5B5C184070470020704769
S3150800449858510008EC4F0008A0F16103192B98BF82
S315080044A820387047A0F14103192B98BF2030704770
S315080044B87F299ABF017001206FF02E00704700BF50
S315080044C85AB10A787F2A0AD800B102600021196011
S315080044D85960501A18BF01207047002070476FF0BE
S315080044E82E00704708B5034B5B689B681B6898479E
S315080044F808BD00BF0400002008B50421FFF7F2FF35
S3150800450808BD00BF08B5034B5B689B685B6898479E
S3150800451808BD00BF040000208446002A2AD010F0EF
S31508004528030F04D000F8011B013A23D0F7E7282A1D
S315080045381CD3A2F128022DE9F00F01F0FF0141EA88
S31508004548012141EA014141EA01610B460C460D4643
S315080045580E460F46884689468A468B46A0E8FA0FCD
S31508004568283AFBD2BDE8F00F283203D000F8011B21
S30D08004578013AFBD160467047C9
S315080045802F64656D6F70726F675F6F6C696D6578A4
S315080045905F73746D3332703130332E737265630016
S315080045A02F626F6F746C6F672E747874000000004A
S315080045B0433A2F576F726B2F736F66747761726504
S315080045C02F4F70656E424C542F5461726765742F75
S315080045D044656D6F2F41524D434D335F53544D33F0
S315080045E03246315F4F6C696D65785F53544D33328F
S315080045F0503130335F43726F7373776F726B732FFB
S31508004600426F6F742F6964652F2E2E2F6D61696E48
S315080046102E630000433A2F576F726B2F736F6674C1
S31508004620776172652F4F70656E424C542F546172D4
S315080046306765742F44656D6F2F41524D434D335F47
S3150800464053544D333246315F4F6C696D65785F530D
S31508004650544D3332503130335F43726F7373776F13
S31508004660726B732F426F6F742F6964652F2E2E2F0E
S31508004670766563746F72732E63000000433A2F5792
S315080046806F726B2F736F6674776172652F4F7065E3
S315080046906E424C542F5461726765742F44656D6F72
S315080046A02F41524D434D335F53544D333246315F9C
S315080046B04F6C696D65785F53544D333250313033E2
S315080046C05F43726F7373776F726B732F426F6F747A
S315080046D02F6964652F2E2E2F2E2E2F2E2E2F2E2E3F
S315080046E02F536F757263652F41524D434D335F5398
S315080046F0544D333246312F63616E2E63000000003D
S3150800470005020602060307030803090309040A0447
S315080047100B040C040C050D050E050F050F061006F7
S3150800472010071008006000080020000003000000C1
S3150800473000800008002000000400000000A0000817
S31508004740002000000500000000C00008002000004E
S315080047500600000000E00008002000000700000036
S3150800476000000108002000000800000000200108E1
S315080047700020000009000000004001080020000099
S315080047800A00000000600108002000000B0000007D
S3150800479000800108002000000C00000000A00108AD
S315080047A0002000000D00000000C0010800200000E5
S315080047B00E00000000E00108002000000F000000C5
S315080047C0433A2F576F726B2F736F667477617265F2
S315080047D02F4F70656E424C542F5461726765742F63
S315080047E044656D6F2F41524D434D335F53544D33DE
S315080047F03246315F4F6C696D65785F53544D33327D
S31508004800503130335F43726F7373776F726B732FE8
S31508004810426F6F742F6964652F2E2E2F2E2E2F2E22
S315080048202E2F2E2E2F536F757263652F41524D43CF
S315080048304D335F53544D333246312F756172742EA2
S31508004840630000004F70656E424C5400303A000019
S31508004850433A2F576F726B2F736F66747761726561
S315080048602F4F70656E424C542F5461726765742FD2
S3150800487044656D6F2F41524D434D335F53544D334D
S315080048803246315F4F6C696D65785F53544D3332EC
S31508004890503130335F43726F7373776F726B732F58
S315080048A0426F6F742F6964652F2E2E2F2E2E2F2E92
S315080048B02E2F2E2E2F536F757263652F66696C65C2
S315080048C02E6300004669726D7761726520757064A3
S315080048D061746520726571756573742064657465A5
S315080048E0637465640A0D00004F70656E696E672013
S315080048F06669726D776172652066696C6520666F98
S31508004900722072656164696E672E2E2E00000000A3
S315080049104552524F520A0D004F4B0A0D0000000037
S315080049205374617274696E67207468652070726F5B
S315080049306772616D6D696E672073657175656E6303
S31508004940650A0D0050617273696E67206669726D3B
S31508004950776172652066696C6520746F206465747A
S3150800496065637420657261736520626C6F636B732F
S315080049702E2E2E0045726173696E672000000000B6
S315080049802062797465732066726F6D206D656D6F30
S3150800499072792061742030780000000052656164E5
S315080049A0696E67206C696E652066726F6D20666930
S315080049B06C652E2E2E4552524F520A0D00000000ED
S315080049C0496E76616C696420636865636B73756D9F
S315080049D020666F756E642E2E2E4552524F520A0D62
S315080049E00000000050726F6772616D6D696E672016
S315080049F00000000020627974657320746F206D656D
S31508004A006D6F72792061742030780000577269746E
S31508004A10696E672070726F6772616D20636865637F
S31508004A206B73756D2E2E2E00436C6F73696E67203F
S31508004A306669726D776172652066696C650A0D0034
S31508004A404669726D77617265207570646174652058
S31508004A507375636365737366756C6C7920636F6DC4
S31508004A60706C657465640A0D00000000222A3A3CE1
S31508004A703E3F7C7F000000002B2C3B3D5B5D000029
S31508004A80809A45418E418F804545454949498E8FD3
S31508004A909092924F994F555559999A9B9C9D9E9FD6
S31508004AA041494F55A5A5A6A7A8A9AAABACADAEAFD7
S31508004AB0B0B1B2B3B4B5B6B7B8B9BABBBCBDBEBF70
S31508004AC0C0C1C2C3C4C5C6C7C8C9CACBCCCDCECF60
S31508004AD0D0D1D2D3D4D5D6D7D8D9DADBDCDDDEDF50
S31508004AE0E0E1E2E3E4E5E6E7E8E9EAEBECEDEEEF40
S31508004AF0F0F1F2F3F4F5F6F7F8F9FAFBFCFDFEFF30
S31508004B0001030507090E10121416181C1E000000D2
S31508004B10C700FC00E900E200E400E000E500E70069
S31508004B20EA00EB00E800EF00EE00EC00C400C50068
S31508004B30C900E600C600F400F600F200FB00F90022
S31508004B40FF00D600DC00A200A300A500A720920162
S31508004B50E100ED00F300FA00F100D100AA00BA0066
S31508004B60BF001023AC00BD00BC00A100AB00BB0019
S31508004B70912592259325022524256125622556250A
S31508004B8055256325512557255D255C255B2510256B
S31508004B90142534252C251C2500253C255E255F2556
S31508004BA05A25542569256625602550256C256725CF
S31508004BB068256425652559255825522553256B25CD
S31508004BC06A2518250C25882584258C259025802579
S31508004BD0B103DF009303C003A303C303B500C403F3
S31508004BE0A6039803A903B4031E22C603B503292204
S31508004BF06122B1006522642220232123F70048227E
S31508004C00B0001922B7001A227F20B200A025A00002
S31508004C107D1D0100632C001E9601A01E5A01001F6F
S31508004C200806101F0606201F0806301F0806401F24
S31508004C300606511F0700591F521F5B1F541F5D1F91
S31508004C40561F5F1F601F0806701F0E00BA1FBB1F86
S31508004C50C81FC91FCA1FCB1FDA1FDB1FF81FF91F82
S31508004C60EA1FEB1FFA1FFB1F801F0806901F080686
S31508004C70A01F0806B01F0400B81FB91FB21FBC1F2B
S31508004C80CC1F0100C31FD01F0206E01F0206E51F46
S31508004C900100EC1FF21F0100FC1F4E21010032210A
S31508004CA070211002842101008321D0241A05302C9A
S31508004CB02F04602C0201672C0601752C0201802C3A
S31508004CC06401002D260841FF1A03000061001A033B
S31508004CD0E0001703F8000703FF0001007801000150
S31508004CE0300132010601390110014A012E0179010C
S31508004CF0060180014D00430281018201820184017F
S31508004D00840186018701870189018A018B018B014C
S31508004D108D018E018F0190019101910193019401FA
S31508004D20F60196019701980198013D029B019C01A5
S31508004D309D0120029F01A001A001A201A201A401D8
S31508004D40A401A601A701A701A901AA01AB01AC010B
S31508004D50AC01AE01AF01AF01B101B201B301B301BC
S31508004D60B501B501B701B801B801BA01BB01BC016B
S31508004D70BC01BE01F701C001C101C201C301C401E2
S31508004D80C501C401C701C801C701CA01CB01CA01CF
S31508004D90CD011001DD0101008E01DE011201F301D2
S31508004DA00300F101F401F401F801280122021201BD
S31508004DB03A020900652C3B023B023D02662C3F0283
S31508004DC040024102410246020A01530240008101A3
S31508004DD08601550289018A0158028F015A029001FB
S31508004DE05C025D025E025F02930161026202940147
S31508004DF06402650266026702970196016A02622CDE
S31508004E006C026D026E029C01700271029D017302B2
S31508004E1074029F0176027702780279027A027B028F
S31508004E207C02642C7E027F02A60181028202A9010D
S31508004E308402850286028702AE014402B101B201EC
S31508004E4045028D028E028F0290029102B7017B0302
S31508004E500300FD03FE03FF03AC0304008603880377
S31508004E6089038A03B1031103C2030200A303A30340
S31508004E70C4030803CC0303008C038E038F03D803F3
S31508004E801801F2030A00F903F303F403F503F60322
S31508004E90F703F703F903FA03FA033004200350046F
S31508004EA01007600422018A043601C1040E01CF04EA
S31508004EB00100C004D0044401610526040000000076
S31508004EC04A616E00466562004D617200417072006B
S31508004ED04D6179004A756E004A756C004175670028
S31508004EE0536570004F6374004E6F76004465630027
S31508004EF0000000002E00000073756363657373007D
S31508004F00646F6D61696E206572726F7200000000D1
S31508004F10696C6C6567616C2073657175656E636530
S31508004F20206572726F72000072616E676520657225
S31508004F30726F7200636F7272757074206865617043
S31508004F40000000006E6F206D656D6F7279000000BD
S31508004F50696E76616C696420617267756D656E74D9
S31508004F6000000000756E6B6E6F776E206572726F4B
S31508004F70720000003B00000043000000504F5349F8
S31508004F805800000025412C202542202523642C208A
S31508004F9025592C2025483A254D3A2553000000006E
S31508004FA0256D2F25642F25790000000025592D250C
S31508004FB06D2D25640000000025493A254D3A2573D4
S31508004FC02025700025483A254D00000025412C2053
S31508004FD02542202523642C202559000000000000C6
S31508004FE0784F000860500008B850000800070320F2
S31508004FF004170201085710408000000053756E64BC
S315080050006179004D6F6E64617900547565736461EA
S3150800501079005765646E65736461790054687572C2
S3150800502073646179004672696461790053617475C5
S31508005030726461790000000053756E004D6F6E0052
S3150800504054756500576564005468750046726900B2
S315080050505361740000000000414D00504D000000EF
S31508005060F44E0008DC4F0008DC4F0008DC4F00084F
S31508005070DC4F0008DC4F0008DC4F0008DC4F000856
S31508005080DC4F0008DC4F0008FFFFFFFFFFFFFFFFB4
S31508005090FFFFFFFFFFFF0000FC4F00083850000825
S315080050A0D8500008C04E0008585000084C51000857
S315080050B04051000830510008514400086D4400086A
S315080050C07944000885440008A1440008AD44000856
S315080050D0B9440008C94400084A616E7561727900CE
S315080050E04665627275617279004D61726368004146
S315080050F07072696C004D6179004A756E65004A7573
S315080051006C79004175677573740053657074656DC5
S31508005110626572004F63746F626572004E6F7665E2
S315080051206D62657200446563656D626572000000B4
S315080051302561202562202565202554202559000053
S3150800514025483A254D3A255300000000256D2F25A0
S31508005150642F257900000000202020202020202010
S3150800516020682828282820202020202020202020C9
S315080051702020202020202020481010101010101069
S315080051801010101010101010848484848484848471
S315080051908484101010101010108181818181810182
S315080051A001010101010101010101010101010101E1
S315080051B00101011010101010108282828282820270
S315080051C002020202020202020202020202020202B1
S30D080051D0020202101010102063
S315080051D801040000E04F0008E04F0008E04F00080F
S30D080051E8E04F0008E04F000843
S70508000151A0
